:020000040800F2
:100000000000052409110008150F0008170F00084B
:10001000190F00081B0F00081D0F0008000000004A
:100020000000000000000000000000001F0F00089A
:10003000210F000800000000230F0008250F000812
:1000400059110008591100085911000859110008E8
:1000500059110008591100085911000859110008D8
:1000600059110008591100085911000859110008C8
:1000700059110008591100085911000859110008B8
:100080005911000859110008591100082D0F0008D6
:10009000591100083D0F00085911000859110008B6
:1000A0005911000859110008591100085911000888
:1000B0005911000859110008591100085911000878
:1000C0005911000859110008591100085911000868
:1000D000591100084D0F0008591100085911000866
:1000E00059110008591100080000000059110008BA
:1000F0005911000859110008591100085911000838
:100100005911000859110008591100085911000827
:100110005911000859110008591100085911000817
:100120005911000859110008591100085911000807
:1001300059110008591100085911000859110008F7
:1001400000000000000000000000000000000000AF
:1001500059110008591100085911000859110008D7
:1001600059110008591100085911000859110008C7
:100170005911000859110008591100080000000029
:1001800059110008591100085911000859110008A7
:100190005911000859110008591100085911000897
:1001A00059110008591100085911000800000000F9
:1001B0005911000859110008591100085911000877
:1001C000591100085911000800000000000000004B
:1001D00000000000000000005911000800000000AD
:1001E000000000000000000000000000000000000F
:1001F000000000000000000059110008591100081B
:100200005911000859110008000000005911000898
:100210005911000859110008591100085911000816
:1002200059110008000000005911000800000000EA
:100230005911000859110008000000005911000868
:1002400059110008591100085911000859110008E6
:1002500059110008591100085911000859110008D6
:1002600059110008591100085911000859110008C6
:100270005911000859110008591100080000000028
:1002800059110008591100085911000859110008A6
:10029000000000005911000859110008000000007A
:1002A00000000000591100085911000859110008F8
:1002B0005911000859110008591100085911000876
:0C02C000591100085911000859110008DC
:1002CC0010B5054C237833B9044B13B10448AFF384
:1002DC0000800123237010BD3C04002400000000AA
:1002EC008051000808B5034B1BB103490348AFF319
:1002FC00008008BD0000000040040024805100086C
:10030C0080F0004002E000BF81F0004142001FBFBE
:10031C005FEA410392EA030F7FEA226C7FEA236CC7
:10032C006AD04FEA1262D2EB1363C1BFD2184140BC
:10033C0048404140B8BF5B42192B88BF704710F052
:10034C00004F40F4000020F07F4018BF404211F0F5
:10035C00004F41F4000121F07F4118BF494292EA5D
:10036C00030F3FD0A2F1010241FA03FC10EB0C0089
:10037C00C3F1200301FA03F100F0004302D5494216
:10038C0060EB4000B0F5000F13D3B0F1807F06D3C3
:10039C0040084FEA310102F10102FE2A51D2B1F1BB
:1003AC00004F40EBC25008BF20F0010040EA0300B0
:1003BC007047490040EB0000013A28BFB0F5000F30
:1003CC00EDD2B0FA80FCACF1080CB2EB0C0200FAE6
:1003DC000CF0AABF00EBC25052421843BCBFD04035
:1003EC001843704792F0000F81F4000106BF80F4AF
:1003FC0000000132013BB5E74FEA41037FEA226C72
:10040C0018BF7FEA236C21D092EA030F04D092F03C
:10041C00000F08BF0846704790EA010F1CBF002070
:10042C00704712F07F4F04D1400028BF40F00040CD
:10043C00704712F100723CBF00F50000704700F0ED
:10044C00004343F0FE4040F4000070477FEA226214
:10045C0016BF08467FEA23630146420206BF5FEAE5
:10046C00412390EA010F40F4800070474FF00003E5
:10047C0004E000BF10F0004348BF40425FEA000CAC
:10048C0008BF704743F0964301464FF000001CE054
:10049C0050EA010208BF70474FF000030AE000BFAA
:1004AC0050EA010208BF704711F0004302D54042E8
:1004BC0061EB41015FEA010C02BF8446014600205A
:1004CC0043F0B64308BFA3F18053A3F50003BCFA75
:1004DC008CF2083AA3EBC25310DB01FA02FC634422
:1004EC0000FA02FCC2F12002BCF1004F20FA02F229
:1004FC0043EB020008BF20F00100704702F120021C
:10050C0001FA02FCC2F1200250EA4C0021FA02F27C
:10051C0043EB020008BF20EADC7070474FF0FF0C81
:10052C001CEAD0521EBF1CEAD15392EA0C0F93EA7C
:10053C000C0F6FD01A4480EA010C400218BF5FEA1E
:10054C0041211ED04FF0006343EA501043EA511191
:10055C00A0FB01310CF00040B1F5000F3EBF49008B
:10056C0041EAD3715B0040EA010062F17F02FD2A8F
:10057C001DD8B3F1004F40EBC25008BF20F0010072
:10058C00704790F0000F0CF0004C08BF49024CEA89
:10059C00502040EA51207F3AC2BFD2F1FF0340EA1B
:1005AC00C250704740F400004FF00003013A5DDC8C
:1005BC0012F1190FDCBF00F000407047C2F10002CD
:1005CC00410021FA02F1C2F1200200FA02FC5FEABA
:1005DC00310040F1000053EA4C0308BF20EADC7004
:1005EC00704792F0000F00F0004C02BF400010F476
:1005FC00000F013AF9D040EA0C0093F0000F01F023
:10060C00004C02BF490011F4000F013BF9D041EA44
:10061C000C018FE70CEAD15392EA0C0F18BF93EA46
:10062C000C0F0AD030F0004C18BF31F0004CD8D170
:10063C0080EA010000F00040704790F0000F17BFF7
:10064C0090F0004F084691F0000F91F0004F14D03D
:10065C0092EA0C0F01D142020FD193EA0C0F03D195
:10066C004B0218BF084608D180EA010000F0004098
:10067C0040F0FE4040F40000704740F0FE4040F473
:10068C00400070474FF0FF0C1CEAD0521EBF1CEA12
:10069C00D15392EA0C0F93EA0C0F69D0A2EB030230
:1006AC0080EA010C49024FEA402037D04FF08053CA
:1006BC0043EA111143EA10130CF000408B4238BF8F
:1006CC005B0042F17D024FF4000C8B4224BF5B1A9D
:1006DC0040EA0C00B3EB510F24BFA3EB510340EAEB
:1006EC005C00B3EB910F24BFA3EB910340EA9C0099
:1006FC00B3EBD10F24BFA3EBD10340EADC001B0109
:10070C0018BF5FEA1C1CE0D1FD2A3FF650AF8B42AC
:10071C0040EBC25008BF20F0010070470CF0004CB9
:10072C004CEA50207F32C2BFD2F1FF0340EAC250E4
:10073C00704740F400004FF00003013A37E792F0A5
:10074C00000F00F0004C02BF400010F4000F013A03
:10075C00F9D040EA0C0093F0000F01F0004C02BFFE
:10076C00490011F4000F013BF9D041EA0C0195E767
:10077C000CEAD15392EA0C0F08D142027FF47DAF00
:10078C0093EA0C0F7FF470AF084676E793EA0C0FF0
:10079C0004D14B023FF44CAF08466EE730F0004CEE
:1007AC0018BF31F0004CCAD130F000427FF45CAF7E
:1007BC0031F000437FF43CAF5FE700BF42000ED244
:1007CC00B2F1FE4F0BD34FF09E03B3EB126209D480
:1007DC004FEA002343F0004323FA02F070474FF036
:1007EC000000704712F1610F01D1420202D14FF0AB
:1007FC00FF3070474FF00000704700BF53B94AB943
:10080C00002908BF00281CBF4FF0FF314FF0FF300C
:10081C0000F06CB9ADF1080C6DE904CE00F006F8EF
:10082C00DDF804E0DDE9022304B070472DE9F04760
:10083C00089E0D4604468E46002B40F082808A426C
:10084C00174646D9B2FA82F24AB1C2F1200105FA32
:10085C0002F320FA01F1974041EA030E94404FEA6B
:10086C001748230CBEFBF8FCB9B208FB1CEE43EA9C
:10087C000E430CFB01F098420AD9FB180CF1FF3522
:10088C0080F01681984240F21381ACF1020C3B448B
:10089C001B1AA4B2B3FBF8F008FB103344EA034470
:1008AC0000FB01F1A14209D93C1900F1FF3380F0A2
:1008BC000181A14240F2FE8002383C44641A40EAB5
:1008CC000C4000211EB1D4400023C6E90043BDE812
:1008DC00F08702B9FFDEB2FA82F2002A4FD1CB1BAD
:1008EC004FEA174E1FFA87F80121B3FBFEFC250CCB
:1008FC000EFB1C3345EA034508FB0CF3AB4207D94E
:10090C007D190CF1FF3002D2AB4200F2E780844635
:10091C00ED1AA3B2B5FBFEF00EFB105543EA0544ED
:10092C0008FB00F8A04507D93C1900F1FF3302D2AF
:10093C00A04500F2D7801846A4EB080440EA0C400E
:10094C00C0E78B4208D9002E00F0AF800021C6E929
:10095C0000050846BDE8F087B3FA83F100294BD1B6
:10096C00AB4202D3824200F2B780841A65EB0303D8
:10097C0001209E46002EAAD0C6E9004EA7E7C2F180
:10098C00200C01FA02F3974020FA0CF04FEA174EB4
:10099C0021FA0CFC1843BCFBFEF1050C0EFB11CC30
:1009AC001FFA87F845EA0C4501FB08F3AB4204FA41
:1009BC0002F409D97D1901F1FF3C80F08B80AB4228
:1009CC0040F2888002393D44EB1A85B2B3FBFEF04D
:1009DC000EFB103345EA034500FB08F3AB4207D985
:1009EC007D1900F1FF3C71D2AB426FD902383D4406
:1009FC00EB1A40EA014178E7C1F1200C8B4022FA56
:100A0C000CF71F4320FA0CF405FA01F34FEA174ECA
:100A1C0025FA0CF51C43230CB5FBFEF91FFA87F8DD
:100A2C000EFB195543EA054509FB08FAAA4502FADB
:100A3C0001F200FA01F308D97D1909F1FF3047D210
:100A4C00AA4545D9A9F102093D44A5EB0A05A4B272
:100A5C00B5FBFEF00EFB105544EA054400FB08F80C
:100A6C00A04507D93C1900F1FF352DD2A0452BD953
:100A7C0002383C4440EA0940A4EB0804A0FB02897C
:100A8C004C45C6464D4619D316D05EB1B3EB0E029B
:100A9C0064EB050404FA0CFCCA404CEA0202CC409C
:100AAC00C6E900240021BDE8F087314630460EE748
:100ABC00AC46EDE6184601E74345E6D2B8EB020E2C
:100ACC0069EB07050138E0E72846D3E760468FE776
:100ADC008146BAE7614677E708464BE7ACF1020C72
:100AEC003D4415E702383C4426E700BF704700BF81
:100AFC00844641EA000313F003036DD1403A41D31D
:100B0C0051F8043B40F8043B51F8043B40F8043BDB
:100B1C0051F8043B40F8043B51F8043B40F8043BCB
:100B2C0051F8043B40F8043B51F8043B40F8043BBB
:100B3C0051F8043B40F8043B51F8043B40F8043BAB
:100B4C0051F8043B40F8043B51F8043B40F8043B9B
:100B5C0051F8043B40F8043B51F8043B40F8043B8B
:100B6C0051F8043B40F8043B51F8043B40F8043B7B
:100B7C0051F8043B40F8043B51F8043B40F8043B6B
:100B8C00403ABDD2303211D351F8043B40F8043B0B
:100B9C0051F8043B40F8043B51F8043B40F8043B4B
:100BAC0051F8043B40F8043B103AEDD20C3205D31B
:100BBC0051F8043B40F8043B043AF9D2043208D013
:100BCC00D2071CBF11F8013B00F8013B01D30B8885
:100BDC0003806046704700BF082A13D38B078DD063
:100BEC0010F003038AD0C3F10403D21ADB071CBF35
:100BFC0011F8013B00F8013B80D331F8023B20F89F
:100C0C00023B7BE7043AD9D3013A11F8013B00F8D7
:100C1C00013BF9D20B7803704B7843708B7883705F
:100C2C006046704700B58BB00B466A46402101F018
:100C3C006DF820B99DF80E000BB05DF804FB002098
:100C4C00FAE7000008B502490248FFF7EBFF08BDC0
:100C5C00580400246004002411F0010F07D008B5DB
:100C6C00034B984200D008BDFFF7ECFFFBE7704741
:100C7C006004002408B51548154B036000238360FD
:100C8C00C36003744374837418224261012282612D
:100C9C000221C161016242628262C26202634363E9
:100CAC008263C36320210164042242648364C264AE
:100CBC00036542658365C36501664366826600F021
:100CCC00DBFE00B908BD00F0ABF8FBE760040024C4
:100CDC0000A0004010B5B6B004460021319132910D
:100CEC00339134913591B82202A804F083F922682B
:100CFC00264B9A4201D036B010BD4FF4004200236F
:100D0C00CDE902234FF080531D9302A802F046FA5E
:100D1C00002837D11E4BD3F8EC2042F48072C3F874
:100D2C00EC20D3F8EC2002F480720092009AD3F8F5
:100D3C00E02042F00102C3F8E020D3F8E03003F0E9
:100D4C0001030193019B4FF4C0533193022332935F
:100D5C000024339434940923359331A90D4801F0C0
:100D6C005FFA22462146132000F06CFA132000F0A3
:100D7C009BFA22462146152000F064FA152000F05B
:100D8C0093FAB8E700F04CF8C4E700BF00A00040AD
:100D9C00004402580000025830B589B00024039476
:100DAC0004940594069407941B4BD3F8E02042F06E
:100DBC008002C3F8E020D3F8E02002F08002009219
:100DCC00009AD3F8E02042F00102C3F8E020D3F8F7
:100DDC00E02002F001020192019AD3F8E02042F0E7
:100DEC000202C3F8E020D3F8E03003F002030293D0
:100DFC00029B0A4D22468021284601F001FB8023EC
:100E0C000393012304930594069403A9284601F047
:100E1C0007FA09B030BD00BF004402580000025868
:100E2C0072B6FEE710B59CB04C22002109A804F064
:100E3C00E1F82022002101A804F0DCF8022001F0E6
:100E4C00E5FA00230093204B9A6922F440429A6100
:100E5C009B6903F440430093009B1B4B9B6913F469
:100E6C00005FFAD00222099201200C9040230D93CE
:100E7C00129200231393042114911E24159416909E
:100E8C00179118920C2219921A931B9309A801F02E
:100E9C00E7FAA0B93F2301930321029100230393A6
:100EAC00082304934023059306934FF48062079222
:100EBC00089301A801F0D6FE18B91CB010BDFFF7BD
:100ECC00AFFFFFF7ADFF00BF0048025808B500F0B8
:100EDC0067F9FFF7A7FFFFF75FFFFFF7CBFE00F007
:100EEC0083F8FEE782B0074BD3F8F42042F00202FD
:100EFC00C3F8F420D3F8F43003F002030193019B00
:100F0C0002B0704700440258FEE7FEE7FEE7FEE73A
:100F1C00FEE770477047704708B500F06FF908BDE1
:100F2C0008B5024800F0ECFF08BD00BF60040024C7
:100F3C0008B5024800F0E4FF08BD00BF60040024BF
:100F4C0008B5024803F010F908BD00BF00050024E5
:100F5C001E4B1B6803F00F03062B06D81B4A1368A5
:100F6C0023F00F0343F007031360194B1A6842F088
:100F7C0001021A6000221A611968164A0A401A60A6
:100F8C00124B1B6813F0080F06D0104A136823F09D
:100F9C000F0343F0070313600D4B00229A61DA61D3
:100FAC001A620D4999620D49D9620D4919635A6348
:100FBC009963DA6319645A64196821F48021196001
:100FCC001A66084B43F2D2021A6070470020005296
:100FDC00004402587FEDF6EA000202020000FF0115
:100FEC00800201010040005208B51748174B0360FE
:100FFC004FF4E133436000238360C36003610C2230
:10100C0042618361C36103624362836203F009FF3F
:10101C0070B900210C4803F07FFF60B900210A4829
:10102C0003F09FFF50B9084803F057FF48B908BDBB
:10103C00FFF7F6FEEDE7FFF7F3FEEFE7FFF7F0FE45
:10104C00F1E7FFF7EDFEF2E7000500240010014088
:10105C0010B5B6B0044600213191329133913491E0
:10106C003591B82202A803F0C5FF2268204B9A42A2
:10107C0001D036B010BD01220023CDE9022300239C
:10108C00209302A802F08AF878BB1A4BD3F8F02010
:10109C0042F01002C3F8F020D3F8F02002F0100256
:1010AC000092009AD3F8E02042F00202C3F8E0204C
:1010BC00D3F8E03003F002030193019B4FF440435B
:1010CC0031930223329300243394349404233593C4
:1010DC0031A9094801F0A4F822462146252000F048
:1010EC00B1F8252000F0E0F8C3E7FFF799FECCE754
:1010FC00001001400044025800040258DFF834D0BC
:10110C00FFF726FF0C480D490D4A002302E0D45886
:10111C00C4500433C4188C42F9D30A4A0A4C002335
:10112C0001E013600432A242FBD303F03FFFFFF750
:10113C00CDFE704700000524000000243C04002470
:10114C00445200083C040024BC050024FEE70000C7
:10115C00104B1B780BB90120704710B504464FF4A7
:10116C007A70B0FBF3F30C4A1068B0FBF3F000F0AC
:10117C00A9F868B90F2C01D901200AE000222146F8
:10118C004FF0FF3000F05EF8044B1C60002000E0D4
:10119C00012010BD08000024000000240C000024D5
:1011AC0010B5032000F03CF801F050FC0F498B699E
:1011BC00C3F303230E4AD35C03F01F03D8408B699F
:1011CC0003F00F03D35C03F01F0320FA03F3094A67
:1011DC001360094B18600F20FFF7BAFF10B1012400
:1011EC00204610BD0446FFF77DFEF9E70044025887
:1011FC00E45100080400002400000024034B1B7879
:10120C00034A11680B441360704700BF08000024A8
:10121C0094050024014B1868704700BF9405002406
:10122C000649CB6823F4E0631B041B0C000200F49A
:10123C00E0600343024A1A43CA60704700ED00E0C5
:10124C000000FA0530B4154BDB68C3F30223C3F17D
:10125C000704042C28BF04241D1D062D14D9033BA0
:10126C004FF0FF3505FA04F421EA0401994005FA20
:10127C0003F322EA03031943002807DB0901C9B26F
:10128C00074B195430BC70470023E9E700F00F00FE
:10129C000901C9B2034B1954F4E700BF00ED00E09B
:1012AC0000E400E014ED00E0002807DB00F01F0272
:1012BC00400901239340024A42F82030704700BF96
:1012CC0000E100E00138B0F1807F0AD2064B586093
:1012DC00064AF02182F823100020986007221A6039
:1012EC0070470120704700BF10E000E000ED00E007
:1012FC0070B50446FFF78EFF002C00F09181054677
:10130C0094F83530DBB2022B06D0802363650023C2
:10131C0084F83430012070BD23688C498C4A934288
:10132C0018BF8B4230D0183293422DD018329342D2
:10133C002AD01832934227D01832934224D0183234
:10134C00934221D0183293421ED002F5567293422A
:10135C001AD01832934217D01832934214D0183244
:10136C00934211D0183293420ED0183293420BD0C4
:10137C001832934208D01832934205D01A6822F0E2
:10138C000E021A60266809E01A6822F01E021A6022
:10139C002268536923F080035361266823686B49E4
:1013AC006B4A934218BF8B4242D0183293423FD0C3
:1013BC00183293423CD01832934239D018329342AF
:1013CC0036D01832934233D01832934230D002F5D3
:1013DC00567293422CD01832934229D01832934231
:1013EC0026D01832934223D01832934220D0183290
:1013FC0093421DD0183293421AD01832934217D010
:10140C00544A934214D01432934211D01432934262
:10141C000ED0143293420BD01432934208D01432B3
:10142C00934205D01432934202D01432934204D129
:10143C00226E136823F48073136023684349444A73
:10144C00934218BF8B422FD0183293422CD01832B3
:10145C00934229D01832934226D01832934223D08B
:10146C001832934220D0183293421DD002F5567296
:10147C00934219D01832934216D01832934213D09B
:10148C001832934210D0183293420DD01832934236
:10149C000AD01832934207D01832934204D01A68FB
:1014AC0022F001021A6003E01A6822F001021A60AD
:1014BC00336813F0010F0ED0FFF7ACFE431B052B66
:1014CC00F6D920236365032384F83530002384F890
:1014DC00343001201FE723681C491D4A934218BF72
:1014EC008B4239D01832934236D01832934233D0D3
:1014FC001832934230D0183293422DD01832934286
:10150C002AD01832934227D002F55672934223D038
:10151C001832934220D0183293421DD01832934285
:10152C001AD01832934217D01832934214D0183272
:10153C00934211D0183293420ED0A16DE36D03F09B
:10154C001F02012393404B600DE000BF10000240CE
:10155C002800024008540258A16DE36D03F01F02ED
:10156C003F2393408B6023682E492F4A934218BF28
:10157C008B4242D0183293423FD0183293423CD027
:10158C001832934239D01832934236D018329342E3
:10159C0033D01832934230D002F5567293422CD08D
:1015AC001832934229D01832934226D018329342E3
:1015BC0023D01832934220D0183293421DD01832C7
:1015CC0093421AD01832934217D0184A934214D02F
:1015DC001432934211D0143293420ED014329342EF
:1015EC000BD01432934208D01432934205D01432EB
:1015FC00934202D0143293420BD1636EA26E5A60A6
:10160C00E36E33B11A6822F480721A60236F626F32
:10161C005A60012384F83530002084F834007AE6CF
:10162C00012078E6100002402800024008540258BD
:10163C00002800F0298108B5024690F83530DBB25D
:10164C00022B03D080234365012008BD036890481A
:10165C0090498B4218BF83420CBF0121002166D0F8
:10166C003030834263D01830834260D018308342CC
:10167C005DD0183083425AD01830834257D018307E
:10168C00834254D000F55670834250D018308342B8
:10169C004DD0183083424AD01830834247D018308E
:1016AC00834244D01830834241D0183083423ED01C
:1016BC00183083423BD0196821F00E011960136871
:1016CC00A0F5956073498B4218BF83426AD072496A
:1016DC008B4267D018318B4264D018318B4261D069
:1016EC0018318B425ED018318B425BD018318B4253
:1016FC0058D001F556718B4254D018318B4251D0D1
:10170C0018318B424ED018318B424BD018318B4252
:10171C0048D018318B4245D018318B4242D0183109
:10172C008B423FD0196821F0010119603EE0042082
:10173C0082F8350081BB584A93422DD0183293421F
:10174C002AD01832934227D01832934224D0183220
:10175C00934221D0183293421ED002F55672934216
:10176C001AD01832934217D01832934214D0183230
:10177C00934211D0183293420ED0183293420BD0B0
:10178C001832934208D01832934205D01A6822F0CE
:10179C0001021A60002058E71A6822F001021A6050
:1017AC00002052E7196821F00101196013683848CC
:1017BC0038498B4218BF834242D018318B423FD0FC
:1017CC0018318B423CD018318B4239D018318B42B6
:1017DC0036D018318B4233D018318B4230D001F5D2
:1017EC0056718B422CD018318B4229D018318B4238
:1017FC0026D018318B4223D018318B4220D018318F
:10180C008B421DD018318B421AD018318B4217D015
:10181C0022498B4214D014318B4211D014318B429B
:10182C000ED014318B420BD014318B4208D01431B2
:10183C008B4205D014318B4202D014318B4217D11C
:10184C00116E0B6823F480730B60906DD36D03F0F5
:10185C001F0101238B404360536E916E5960D36E10
:10186C0033B1196821F480711960136F516F59608D
:10187C00012382F83530002382F83430136D2BB1FC
:10188C00104698470020E0E6012070470020DCE677
:10189C001000024028000240400002400854025848
:1018AC0030B4446B0268D2F88410704B194041EA92
:1018BC008401C2F884100268D2F8841021F47F01EC
:1018CC00856B41EA0541C2F88410826B224404689E
:1018DC00D4F88810194041EA8201C4F888100468D1
:1018EC00D4F8881021F4FE01C56B41EA0541C4F817
:1018FC008810C16B02EB41020468D4F8A0101940A7
:10190C0041EA8201C4F8A0100468D4F8A01021F4B4
:10191C00FE01056C41EA0541C4F8A010046C416C51
:10192C0001FB04240268D2F8B010194041EA84018A
:10193C00C2F8B0100268D2F8B01021F4FE01856C28
:10194C0041EA0541C2F8B010826CC16C01FB024443
:10195C000268D2F8AC10194041EA8401C2F8AC100C
:10196C00026D416D01FB02420468D4F8F01019407D
:10197C0041EA8201C4F8F0100468D4F8F01021F4A4
:10198C007C11856D41EA0541C4F8F010816D02EBC4
:10199C0041020468D4F8C0100B4043EA8202C4F838
:1019AC00C0200268D2F8C03023F47C13C16D43EA26
:1019BC000143C2F8C0300268D2F8C03023F07C5327
:1019CC00016E43EA0163C2F8C030436B284A1A44E3
:1019DC009200C266836B02EB83030367C16B03EB5C
:1019EC00C1034367046C416C01FB04F103EB8103FD
:1019FC008367846CC16C01FB04F103EB8103C36747
:101A0C00046D416D01FB04F103EB8103C0F88030E0
:101A1C00816D03EBC103C0F88430C46D856E05FB8A
:101A2C0004F403EB8403C0F88830016E01FB05F16C
:101A3C0003EB8103C0F890300E498B4207D8D0F8E5
:101A4C00903093420ED9002342F8043BF7E7D0F8CC
:101A5C009C3043F02003C0F89C30032380F898306E
:101A6C00012000E0002030BC704700BF0300FFFFE6
:101A7C00002B0010FCD3004030B595B004464C222E
:101A8C00A04901A8FFF734F8002C00F03881236836
:101A9C009D4A934220D094F898300BB322689369F6
:101AAC0023F010039361FFF7B5FB054623689A6991
:101ABC0012F0080F1AD0FFF7ADFB431B0A2BF5D918
:101ACC00D4F89C3043F00103C4F89C30032384F811
:101ADC009830012015B030BD03F580736360DAE7F0
:101AEC0084F899302046FFF7F5F8D7E79A6942F069
:101AFC0001029A61FFF78EFB054623689A6912F082
:101B0C00010F0FD1FFF786FB401B0A28F5D9D4F83B
:101B1C009C3043F00103C4F89C30032384F89830C4
:101B2C000120D7E79A6942F002029A61237C012BCB
:101B3C0040D02268936943F040039361637C012B8E
:101B4C003ED02268936923F480439361A37C012BDC
:101B5C003CD02268936943F4805393612268936963
:101B6C0023F44073A1680B4393612268936923F0BB
:101B7C00A40393612268136923F010031361E368D3
:101B8C00012B29D0002B2CD0022B00F09B8022683B
:101B9C00936943F0800393612268136943F0100347
:101BAC001361E368032B1CD12268936943F0200373
:101BBC00936116E02268936923F040039361BDE7BB
:101BCC002268936943F480439361BFE72268936969
:101BDC0023F480539361C1E72268936943F00403B3
:101BEC009361A3695A1EE369013B1B0243EA4263FA
:101BFC00226A013A13436269013A216843EA0243BB
:101C0C00CB61A368B3F5407F62D0236E33B12268F9
:101C1C00D2F8C030616E0B43C2F8C030E36D226E57
:101C2C00D3420DD02168D1F8C83023F00703A26E3F
:101C3C0014A800EB820252F84C2C1343C1F8C830A4
:101C4C00236C6BB12168D1F8BC3023F00703626CB4
:101C5C0014A800EB820252F84C2C1343C1F8BC3090
:101C6C00A36C73B12168D1F8BC3023F07003E26C23
:101C7C0014A800EB820252F84C2C43EA0213C1F870
:101C8C00BC30236D73B12168D1F8BC3023F4E06310
:101C9C00626D14A800EB820252F84C2C43EA02232A
:101CAC00C1F8BC302268184B9A4222D00023C4F8E9
:101CBC009430C4F89C30012384F898302046FFF708
:101CCC00EFFD07E72268936943F02003936188E7EF
:101CDC00A36A013BE26A013A43EA0223226B013A0E
:101CEC0043EA0213626A013A216843EA0243CB6079
:101CFC008BE76268936823F003039360D6E70120B7
:101D0C00E8E600BF9851000800A00040F0B490F83D
:101D1C009840E4B2022C40F0D88040290CD04129E4
:101D2C003FD0046D8C4271D8D0F89C3043F0200326
:101D3C00C0F89C300120CFE00468D4F8A05015F412
:101D4C00FE0F0CD0D4F8A45015F07F0F0FD1D0F8A3
:101D5C009C3043F48073C0F89C300120BCE0D0F878
:101D6C009C3043F02003C0F89C300120B4E0D4F840
:101D7C00A450C5F3006C15F0807F06D0D4F8A050A9
:101D8C005FEAD57C01D14FF0000CD4F8A440C4F329
:101D9C000524A444446F456C0CFB05F504EB850449
:101DAC003CE00468D4F8B05015F4FE0F0CD0D4F815
:101DBC00B45015F07F0F0FD1D0F89C3043F48073E2
:101DCC00C0F89C30012087E0D0F89C3043F0200311
:101DDC00C0F89C3001207FE0D4F8B450C5F3006CFF
:101DEC0015F0807F06D0D4F8B0505FEAD57C01D1D5
:101DFC004FF0000CD4F8B440C4F30524A444846F11
:101E0C00C56C0CFB05F504EB850407E0C46F456D50
:101E1C0001FB05F504EB85044FF0000C256805F07B
:101E2C0080455560002D2CD12568C5F38A45156079
:101E3C00256805F000559560256805F0004515618D
:101E4C00A588D561E58805F00F05D560656805F4B2
:101E5C0080155561656805F400159561E57905F007
:101E6C007F0515626568ED0F556204F108050024C5
:101E7C00D6681A4FBE5DA64208D92E5D1E55013498
:101E8C00F6E7256825F060451560D1E740290AD0B2
:101E9C0041290DD01F290FD80268012303FA01F143
:101EAC00C2F8981002E00368C3F8A8C0002013E041
:101EBC000368C3F8B8C0F9E701F01F0102680123F9
:101ECC0003FA01F1C2F89C10F0E7D0F89C3043F013
:101EDC000803C0F89C300120F0BC7047F451000896
:101EEC00704770477047704770477047704770472E
:101EFC00704770477047704770477047704770471E
:101F0C002DE9F04F83B00446B74B1A695B699B0708
:101F1C0003EA8273019303681A6D02F4704A5A6DD6
:101F2C000AEA020A1A6D02F00F095A6D09EA02094F
:101F3C001A6D02F0F0085A6D08EA02081E6D06F0E0
:101F4C0071565A6D16401F6D07F060775A6D174029
:101F5C005D6DD3F850B015F4807F02D01BF4807FF8
:101F6C0064D115F4806F02D01BF4806F67D1019B94
:101F7C00002B74D1BAF1000F7CD1B9F1000F40F0F5
:101F8C008580B8F1000F40F08D8015F4006F03D000
:101F9C001BF4006F40F0928015F4007F03D01BF40B
:101FAC00007F40F0968015F4002F03D01BF4002F17
:101FBC0040F09F8015F4803F03D01BF4803F40F02D
:101FCC00A38015F4802F03D01BF4802F40F0A78042
:101FDC0015F4003F0FD01BF4003F0CD023684FF4D6
:101FEC0000321A65804B00221A61D4F89C3043F001
:101FFC008003C4F89C30002F40F09C804EB12368C5
:10200C001E65B20F784B1A61D4F89C301E43C4F88D
:10201C009C602268754B9A4200F09680D4F89C30F4
:10202C00002B40F0F88003B0BDE8F08F4FF48072C5
:10203C001A656D4B00221A61FFF75BFF91E723686D
:10204C00D3F8DC10D3F8E4204FF480601865664BAD
:10205C000020186111402046FFF747FF87E72368EF
:10206C0000221A6501998A0F5F4B1A612046FFF70F
:10207C0037FF7FE72368C3F850A04FEA9A725A4B98
:10208C001A6151462046FFF72CFF76E72368C3F808
:10209C0050904FEA9972544B1A6149462046FEF70C
:1020AC00DBFD6EE72368C3F850804FEA98724E4B05
:1020BC001A6141462046FFF715FF66E723684FF487
:1020CC0000621A65484B00221A612046FFF70BFF8D
:1020DC0062E72368D3F8D810D3F8E0204FF40070EF
:1020EC001865414B0020186111402046FFF7FCFE9B
:1020FC0059E723684FF400221A653B4B00221A6102
:10210C002046FFF7F3FE55E723684FF480321A653B
:10211C00354B00221A612046FFF7E9FE51E7236890
:10212C004FF480221A65304B00221A612046FFF7CB
:10213C00DFFE4DE723681F65BA0F2B4B1A6139463A
:10214C002046FFF7D8FE59E763689A6812F0030F30
:10215C003FF464AF196A01F00F015A6A186A00F073
:10216C003008586A08EA00081F6A07F4C077586AF2
:10217C0007401E6A06F4FC46586A06401D6A05F4C0
:10218C00F025586A0540D3F82490D3F820A01140CC
:10219C001CD1B8F1000F1ED119F0400F02D01AF06B
:1021AC00400F25D187BB36B163681E62D4F89C30D2
:1021BC001E43C4F89C60002D3FF430AF63681D6271
:1021CC00D4F89C301D43C4F89C5027E71962204674
:1021DC00FFF792FEDDE76368C3F820804146204696
:1021EC00FFF78BFED8E700BF00A8004000A000401E
:1021FC006368D96BDA6B4020186202F03F02090C5D
:10220C002046FFF77BFECDE763681F623946204608
:10221C00FFF775FEC7E72046FFF76CFE03E700BF2C
:10222C00F0B482B000235FE086685F000325BD40F8
:10223C0026EA0506CD68BD4035438560466826EA2A
:10224C0004064D68C5F300149C403443446059E0C7
:10225C00DD08083550F8257003F00704A6000F249C
:10226C00B44027EA04070C69B4403C4340F82540CD
:10227C005CE0092400E00024B4403C4302355C4E91
:10228C0046F825404FF0B0442568D44325EA0206B1
:10229C004F6817F4801F01D042EA05064FF0B04595
:1022AC002E606E6804EA06054F6817F4001F01D013
:1022BC0042EA06054FF0B04675604E4D6D6804EA73
:1022CC0005064F6817F4003F01D042EA0506494D58
:1022DC006E602D682C404E6816F4803F01D042EAA7
:1022EC000504444A146001330A6832FA03F47BD0C3
:1022FC0001249C402240F6D04D6805F00305013DB9
:10230C00012D91D94C6804F00304032C09D0C56845
:10231C005E000324B44025EA04058C68B4402C43C9
:10232C00C4604C6804F00304022C91D005685E0074
:10233C000324B44025EA04054C6804F00304B440BB
:10234C002C4304604C6814F4403FCCD02A4CD4F895
:10235C00F45045F00205C4F8F450D4F8F44004F0FD
:10236C0002040194019C9D08AE1C214C54F826706B
:10237C0003F00304A6000F24B44027EA04071F4C03
:10238C00A0423FF478AF04F58064A0421ED004F55F
:10239C008064A0421CD004F58064A0421AD004F5DD
:1023AC008064A04218D004F58064A04216D004F5D5
:1023BC008064A04214D004F58064A04212D004F5CD
:1023CC000064A0423FF455AF0A2455E7012453E7BB
:1023DC00022451E703244FE704244DE705244BE77F
:1023EC00062449E7072447E702B0F0BC704700BF5A
:1023FC0000040058800000580044025800000258A5
:10240C000AB181617047090481617047134BDB6825
:10241C0013F0040F07D1114BDB6803F00703834261
:10242C001AD00120704710B50C4AD36823F007036B
:10243C001843D060FEF7EEFE0446084B5B6813F4BD
:10244C00005F07D1FEF7E6FE001BB0F57A7FF4D9EA
:10245C00012000E0002010BD002070470048025809
:10246C00002800F0D78238B50446036813F0010F3A
:10247C0025D0AA4A136903F03803926A102B15D0A1
:10248C00182B0FD06368B3F5803F3FD0002B53D18E
:10249C00A24B1A6822F480321A601A6822F4802245
:1024AC001A6038E002F00302022AEBD19B4B1B6846
:1024BC0013F4003F03D06368002B00F0AD82236857
:1024CC0013F0020F00F08880944A1369926A13F09B
:1024DC0038035AD0182B55D0E368002B00F0A98094
:1024EC008E490A6822F0190213430B60FEF792FE24
:1024FC0005468A4B1B6813F0040F40F09180FEF7E1
:10250C0089FE401B0228F4D903208CE2834A13680D
:10251C0043F48033136063682BB3FEF77BFE0546F0
:10252C007E4B1B6813F4003FC9D1FEF773FE401BB2
:10253C006428F5D9032076E2B3F5A02F09D0774BA8
:10254C001A6822F480321A601A6822F480221A6007
:10255C00E1E7724B1A6842F480221A601A6842F45E
:10256C0080321A60D7E7FEF755FE05466B4B1B68A9
:10257C0013F4003FA3D0FEF74DFE401B6428F5D9A1
:10258C00032050E212F0030FA6D1644B1B6813F02A
:10259C00040F03D0E368002B00F040825F4A1368FD
:1025AC0023F01903E1680B431360FEF733FE054675
:1025BC005A4B1B6813F0040F06D1FEF72BFE401B81
:1025CC000228F5D903202EE2544A536823F0FE4327
:1025DC00216943EA01635360236813F0100F51D053
:1025EC004E4A136903F03803926A082B39D0182B22
:1025FC0033D0E369002B68D0484A136843F080035A
:10260C001360FEF707FE0546444B1B6813F4807FEE
:10261C0052D1FEF7FFFD401B0228F5D9032002E240
:10262C003E4A536823F0FE43216943EA0163536039
:10263C00D2E73A4A136823F001031360FEF7EAFD70
:10264C000546364B1B6813F0040FC5D0FEF7E2FDB0
:10265C00401B0228F5D90320E5E102F00302012A10
:10266C00C7D12E4B1B6813F4807F03D0E369802BFA
:10267C0040F0D681294AD36823F07C53216A43EA7F
:10268C000163D360236813F0080F49D0636983B3E7
:10269C00224A536F43F001035367FEF7BBFD054617
:1026AC001E4B5B6F13F0020F3AD1FEF7B3FD401BCC
:1026BC000228F5D90320B6E1184AD36823F07C53DD
:1026CC00216A43EA0163D360DCE7144A136823F000
:1026DC0080031360FEF79EFD0546104B1B6813F438
:1026EC00807FCFD0FEF796FD401B0228F5D9032042
:1026FC0099E10A4A536F23F001035367FEF78AFDF1
:10270C000546064B5B6F13F0020F09D0FEF782FDF6
:10271C00401B0228F5D9032085E100BF0044025874
:10272C00236813F0200F29D0A3699BB1A84A136822
:10273C0043F480531360FEF76DFD0546A44B1B68F4
:10274C0013F4005F1AD1FEF765FD401B0228F5D982
:10275C00032068E19E4A136823F480531360FEF74C
:10276C0059FD05469A4B1B6813F4005F06D0FEF723
:10277C0051FD401B0228F5D9032054E1236813F0C6
:10278C00040F21D1636A002B00F04C81904A12692E
:10279C0002F03802182A00F0EA80022B75D08C4A1D
:1027AC00136823F080731360FEF734FD0446884BE6
:1027BC001B6813F0007F00F0D880FEF72BFD001B88
:1027CC000228F4D903202EE1824A136843F4807363
:1027DC001360FEF71FFD05467E4B1B6813F4807FCC
:1027EC0006D1FEF717FD401B6428F5D903201AE12A
:1027FC00A368012B0AD00BBB754B1A6F22F0010298
:10280C001A671A6F22F004021A6704E0704A136FF9
:10281C0043F001031367A36833B3FEF7FBFC0546D3
:10282C006B4B1B6F13F0020FACD1FEF7F3FC401B8C
:10283C0041F288339842F3D90320F4E0052B09D0F8
:10284C00634B1A6F22F001021A671A6F22F004020E
:10285C001A67E0E75E4B1A6F42F004021A671A6FB0
:10286C0042F001021A67D6E7FEF7D4FC0546584B36
:10287C001B6F13F0020F85D0FEF7CCFC401B41F20E
:10288C0088339842F3D90320CDE0514A136823F0E2
:10289C0080731360FEF7BEFC05464D4B1B6813F0AE
:1028AC00007F06D0FEF7B6FC401B0228F5D90320AA
:1028BC00B9E0474B996A484A0A40A16AE06A41EA82
:1028CC0000110A439A62226B013AC2F30802616B4F
:1028DC000139490289B20A43A16B0139090401F497
:1028EC00FE010A43E16B0139090601F0FE410A437E
:1028FC001A63DA6A22F00102DA62596B374A0A402B
:10290C00A16C42EAC1025A63DA6A22F00C02216C11
:10291C000A43DA62DA6A22F00202616C0A43DA6272
:10292C00DA6A42F48032DA62DA6A42F40032DA624B
:10293C00DA6A42F48022DA62DA6A42F00102DA627E
:10294C001A6842F080721A60FEF764FC0446204B51
:10295C001B6813F0007F06D1FEF75CFC001B0228FD
:10296C00F5D903205FE000205DE000205BE0184912
:10297C008A6A086B012B57D002F00303A16A8B42C1
:10298C0054D1C2F30512E36A9A4251D1C0F3080242
:10299C00236B013B9A424DD1C0F34622636B013B42
:1029AC009A4249D1C0F30642A36B013B9A4245D1EE
:1029BC00C0F30660E36B013B984241D1044B5B6B67
:1029CC00C3F3CC03A26C9A420AD100202BE000BFC7
:1029DC0000440258004802580CFCFFFF0700FFFFA0
:1029EC00184AD36A23F00103D362FEF713FC0546A1
:1029FC00FEF710FCA842FBD0124A516B124B0B4055
:102A0C00A16C43EAC1035363D36A43F00103D3625D
:102A1C00002008E001207047012004E0012002E0C2
:102A2C00012000E0002038BD0120FCE70120FAE77E
:102A3C000120F8E70120F6E70120F4E70120F2E796
:102A4C000120F0E7004402580700FFFFF8B57E4B69
:102A5C001B6903F03803102B00F0F280182B10D0F8
:102A6C0013B17A4C2046F8BD774B1B6813F0200F3E
:102A7C0000F0E880744B1868C0F3C100744CC4407B
:102A8C00F0E7714B9D6A05F003059C6AC4F30514CD
:102A9C00D86A00F001005B6BC3F3CC0300FB03F0BE
:102AAC00FDF7E4FC0646002CDCD0012D76D0022D7F
:102ABC0000F0A4800DB32046FDF7D8FC0146654814
:102ACC00FDF7E0FD0446604B186BC0F30800FDF702
:102ADC00CDFC05464FF064513046FDF71FFD014615
:102AEC002846FDF713FC4FF07E51FDF70FFC014615
:102AFC002046FDF713FD044671E0534B1B6813F0A1
:102B0C00200F29D0504F3B68C3F3C1035048D84025
:102B1C00FDF7ACFC05462046FDF7A8FC014628460F
:102B2C00FDF7B0FD0446386BC0F30800FDF79EFCC2
:102B3C0005464FF064513046FDF7F0FC014628463F
:102B4C00FDF7E4FB4FF07E51FDF7E0FB014620461C
:102B5C00FDF7E4FC044642E02046FDF787FC014605
:102B6C003D48FDF78FFD0446374B186BC0F308004A
:102B7C00FDF77CFC05464FF064513046FDF7CEFC6A
:102B8C0001462846FDF7C2FB4FF07E51FDF7BEFB18
:102B9C0001462046FDF7C2FC044620E02046FDF726
:102BAC0065FC01462B48FDF76DFD0446264B186B62
:102BBC00C0F30800FDF75AFC05464FF0645130464F
:102BCC00FDF7ACFC01462846FDF7A0FB4FF07E510B
:102BDC00FDF79CFB01462046FDF7A0FC04461A4B72
:102BEC001B6BC3F34623581CFDF740FC01462046E3
:102BFC00FDF748FDFDF7E2FD044633E72046FDF7FF
:102C0C0035FC01461548FDF73DFD04460E4B186B8F
:102C1C00C0F30800FDF72AFC05464FF0645130461E
:102C2C00FDF77CFC01462846FDF770FB4FF07E510A
:102C3C00FDF76CFB01462046FDF770FC0446CEE721
:102C4C00074C0FE7024C0DE70044025800093D0009
:102C5C000090D0030024744A0024744C20BCBE4B5A
:102C6C0040787D01002800F0328170B50D46044695
:102C7C009B4B1B6803F00F038B420BD2984A1368D3
:102C8C0023F00F030B431360136803F00F038B4205
:102C9C0040F01F81236813F0040F0CD02269914B74
:102CAC009B6903F070039A4205D98E498B6923F016
:102CBC0070031A438A61236813F0080F0CD0626901
:102CCC00884BDB6903F070039A4205D98549CB69BF
:102CDC0023F070031A43CA61236813F0100F0CD051
:102CEC00A269804BDB6903F4E0639A4205D97D4904
:102CFC00CB6923F4E0631A43CA61236813F0200FF5
:102D0C000CD0E269774B1B6A03F070039A4205D929
:102D1C0074490B6A23F070031A430A62236813F098
:102D2C00020F0CD0E2686F4B9B6903F00F039A42C1
:102D3C0005D96C498B6923F00F031A438A61236808
:102D4C0013F0010F41D0674A936923F47063A168B3
:102D5C000B4393616368022B0AD0032B27D0012B02
:102D6C002CD0604A126812F0040F06D10120ADE09D
:102D7C00126812F4003F00F0AE805A490A6922F042
:102D8C00070213430B61FEF745FA0646554B1B69C8
:102D9C0003F038036268B3EBC20F16D0FEF73AFAB1
:102DAC00801B41F288339842F0D903208EE04D4AC3
:102DBC00126812F0007FE0D1012087E0494A1268C6
:102DCC0012F4807FD9D1012080E0236813F0020F28
:102DDC000CD0E268434B9B6903F00F039A4205D277
:102DEC0040498B6923F00F031A438A613C4B1B68E3
:102DFC0003F00F03AB420AD9394A136823F00F03CF
:102E0C002B431360136803F00F03AB4265D12368A7
:102E1C0013F0040F0CD02269324B9B6903F0700342
:102E2C009A4205D22F498B6923F070031A438A61A9
:102E3C00236813F0080F0CD062692A4BDB6903F08E
:102E4C0070039A4205D22749CB6923F070031A43C9
:102E5C00CA61236813F0100F0CD0A269214BDB69F7
:102E6C0003F4E0639A4205D21E49CB6923F4E06374
:102E7C001A43CA61236813F0200F0CD0E269194B76
:102E8C001B6A03F070039A4205D216490B6A23F0B1
:102E9C0070031A430A62FFF7D9FD12498B69C3F319
:102EAC000323114AD35C03F01F03D8408B6903F052
:102EBC000F03D35C03F01F0320FA03F30B4A1360D8
:102ECC000B4B18600B4B1868FEF742F970BD0120D4
:102EDC0070470120FAE70120F8E70120F6E700BF70
:102EEC000020005200440258E45100080400002461
:102EFC00000000240C00002408B5FFF7A7FD0B4AC6
:102F0C009369C3F303230A49CB5C03F01F0320FA34
:102F1C0003F3926902F00F02885C00F01F0023FAA1
:102F2C0000F0044A1060044A136008BD00440258C3
:102F3C00E4510008040000240000002408B5FFF749
:102F4C00DBFF054BDB69C3F30213044AD35C03F0CC
:102F5C001F03D84008BD00BF00440258E4510008CC
:102F6C0008B5FFF7C9FF054BDB69C3F30223044A1D
:102F7C00D35C03F01F03D84008BD00BF00440258C7
:102F8C00E4510008404B9B6A03F00303032B79D0F8
:102F9C0070B505460E463C4A136823F080631360F7
:102FAC00FEF738F90446384B1B6813F0006F06D057
:102FBC00FEF730F9031B022BF5D9032070BD324B01
:102FCC009A6A22F47C32296842EA01329A626A686F
:102FDC00013AC2F30802A9680139490289B20A43CD
:102FEC00E9680139090401F4FE010A432969013930
:102FFC00090601F0FE410A439A63DA6A22F0C00224
:10300C0069690A43DA62DA6A22F02002A9690A4382
:10301C00DA62DA6A22F01002DA62D96B1B4A0A40D1
:10302C00E96942EAC102DA63DA6A42F01002DA6252
:10303C00C6B91A46DB6A43F40023D362124A1368FA
:10304C0043F080631360FEF7E5F804460E4B1B68F3
:10305C0013F0006F14D1FEF7DDF8001B0228F5D930
:10306C000320ABE7012E05D0074AD36A43F40013C3
:10307C00D362E3E7044AD36A43F48013D362DDE7F7
:10308C0000209BE701207047004402580700FFFF17
:10309C00404B9B6A03F00303032B79D070B50546B4
:1030AC000E463C4A136823F080531360FEF7B2F8C7
:1030BC000446384B1B6813F0005F06D0FEF7AAF8E5
:1030CC00031B022BF5D9032070BD324B9A6A22F0F8
:1030DC007C72296842EA01529A626A68013AC2F328
:1030EC000802A9680139490289B20A43E968013921
:1030FC00090401F4FE010A4329690139090601F0AA
:10310C00FE410A431A64DA6A22F4406269690A438E
:10311C00DA62DA6A22F40072A9690A43DA62DA6ABC
:10312C0022F48072DA62596C1B4A0A40E96942EA5D
:10313C00C1025A64DA6A42F48072DA62C6B91A467B
:10314C00DB6A43F48003D362124A136843F0805362
:10315C001360FEF75FF804460E4B1B6813F0005F1C
:10316C0014D1FEF757F8001B0228F5D90320ABE762
:10317C00012E05D0074AD36A43F08073D362E3E78C
:10318C00044AD36A43F40003D362DDE700209BE7D3
:10319C0001207047004402580700FFFFF8B50446B1
:1031AC00016801F000620023134330D0436EB3F585
:1031BC00001F26D00ED8EBB1B3F5801F07D102212A
:1031CC000830FFF7DFFE054645B12E4621E001260B
:1031DC0035461EE0B3F5401F09D10025A84A136DF2
:1031EC0023F44013616E0B431365002611E0012696
:1031FC0035460EE0A24AD36A43F40033D36200256D
:10320C00ECE702212830FFF743FF0546DCE70026F8
:10321C003546216801F480720023134314D0A36D4A
:10322C00042B37D8DFE803F003282F080800944A52
:10323C00D36A43F40033D3627DBB914A136D23F000
:10324C000703A16D0B431365216801F48062002311
:10325C00134336D0D4F8A430B3F5800F55D021D811
:10326C00002B4CD0B3F5001F19D1002104F108003C
:10327C00FFF788FE05461BE0002104F10800FFF76C
:10328C0081FE0546D8E7002104F12800FFF700FF76
:10329C000546D1E701263546D6E72E46D4E701266A
:1032AC0035460EE0B3F5000F02D0B3F5200F20D158
:1032BC0095BB734A936D23F46003D4F8A4100B43AD
:1032CC009365216801F400620023134339D0D4F8CC
:1032DC00A830B3F1007F5CD023D8002B53D0B3F1CE
:1032EC00807F1BD1002104F10800FFF74BFE05463F
:1032FC001DE0B3F5C00FDBD001263546E1E7604A8F
:10330C00D36A43F40033D362D2E7002104F12800DE
:10331C00FFF7BEFE0546CBE72E46D2E70126354623
:10332C000FE0B3F1806F02D0B3F1A06F25D1002D67
:10333C0036D1534A936D23F0E063D4F8A8100B43B5
:10334C009365216801F000720023134331D0E36CC4
:10335C00202B45D029D833B1102B23D1484AD36A1E
:10336C0043F40033D362002D41D1454AD36C23F092
:10337C003003E16C0B43D3641BE0B3F1407FD6D038
:10338C0001263546DDE73E4AD36A43F40033D36267
:10339C00CDE7002104F12800FFF77AFE0546C6E7C9
:1033AC002E46CEE70126354603E0302BDBD0012636
:1033BC003546216801F48052002313432BD0E36D72
:1033CC00B3F5005F4FD017D8002B46D0B3F5805F14
:1033DC000FD1002104F10800FFF7D4FD054611E0E0
:1033EC00022104F10800FFF7CDFD0546BBE72E4690
:1033FC00DFE7012635460EE0B3F5405F02D0B3F5AA
:10340C00804F27D1002D35D11D4A136D23F4E04395
:10341C00E16D0B431365216801F400520023134343
:10342C003BD0236EB3F5003F58D02BD843B1B3F546
:10343C00803F21D1012104F10800FFF7A3FD0546CF
:10344C00002D52D10E4A136D23F4E023216E0B4351
:10345C00136522E001263546DDE7094AD36A43F4B9
:10346C000033D362CEE7002104F12800FFF710FEF1
:10347C000546C7E72E46CEE7012635460DE000BFD0
:10348C0000440258B3F5802FDAD0B3F5A02FD7D073
:10349C00B3F5403FD4D001263546216801F4804273
:1034AC000023134331D0D4F8AC30B3F1005F49D0D2
:1034BC0020D843B1B3F1805F19D1012104F1080088
:1034CC00FFF760FD0546002D43D1954A936D23F01F
:1034DC00E043D4F8AC100B43936516E0012104F1E2
:1034EC002800FFF7D5FD0546AAE72E46D5E70126AD
:1034FC0035460AE0B3F1804FE5D0B3F1A04FE2D0EE
:10350C00B3F1405FDFD001263546216801F400425B
:10351C000023134309D0E36EB3F1805F1BD0B3F1EA
:10352C00005F26D0E3B101263546216801F0807298
:10353C00002313433FD0A36C032B38D8DFE803F0F0
:10354C0027223027012104F12800FFF7A1FD0546B1
:10355C00B9E72E46D9E7724AD36A43F40033D362F3
:10356C0075B96F4A136D23F04053E16E0B4313652D
:10357C00DBE7012104F10800FFF704FD0546EFE746
:10358C002E46D2E7664AD36A43F40033D3628DB930
:10359C00634AD36C23F00303A16C0B43D3640AE09E
:1035AC00022104F10800FFF7EDFC0546EFE70126C8
:1035BC00354600E02E46216801F4800200231343B7
:1035CC0021D1216801F001020023134300F0978000
:1035DC00A36F282B00F29180DFE803F07F8F8F8F91
:1035EC008F8F8F8F798F8F8F8F8F8F8F888F8F8FFC
:1035FC008F8F8F8F7F8F8F8F8F8F8F8F7F8F8F8FEF
:10360C008F8F8F8F7F00474A136843F4807313604A
:10361C00FDF700FE0746434B1B6813F4807F05D172
:10362C00FDF7F8FDC01B6428F5D90325002D4AD100
:10363C003B4B1B6FD4F8B020534013F4407F0CD09D
:10364C00374B1A6F22F44072196F41F480311967AD
:10365C00196F21F4803119671A67D4F8B030B3F5BB
:10366C00807F15D08DBBD4F8B03003F44072B2F526
:10367C00407F1ED02A4A136923F47C5313612849D6
:10368C000B6FD4F8B020C2F30B0213430B6798E70F
:10369C00FDF7C0FD0746224B1B6F13F0020FE1D163
:1036AC00FDF7B8FDC01B41F288339842F3D90325CE
:1036BC00D8E71B48026922F47C521B4901EA131318
:1036CC0013430361DBE72E467BE72E4679E70121A6
:1036DC0004F10800FFF756FC0546F5B9104A536D86
:1036EC0023F03803A16F0B43536508E0012104F16B
:1036FC002800FFF7CDFC0546EFE70126354621688B
:10370C0001F00202002313432AD0636F052B23D848
:10371C00DFE803F0120C1B1212122E46EFE700BF6B
:10372C000044025800480258CFFFFF00012104F169
:10373C000800FFF727FC05468DB9B54A536D23F0F9
:10374C000703616F0B4353650AE0012104F1280064
:10375C00FFF79EFC0546EFE70126354600E02E46B6
:10376C00216801F004020023134323D0D4F89030D5
:10377C00052B1BD8DFE803F0090313090909012104
:10378C0004F10800FFF7FEFB054695B9A04A936DBE
:10379C0023F00703D4F890100B4393650AE0012142
:1037AC0004F12800FFF774FC0546EEE701263546C8
:1037BC0000E02E46216801F020020023134328D09C
:1037CC00D4F88C30B3F1005F44D017D843B1B3F1C7
:1037DC00805F10D1002104F10800FFF7D3FB0546F0
:1037EC00002D3ED18A4A536D23F0E043D4F88C105F
:1037FC000B4353650DE0012635460AE0B3F1804FCB
:10380C00EED0B3F1A04FEBD0B3F1405FE8D001267E
:10381C003546216801F040020023134331D0D4F81F
:10382C009830B3F5006F4FD020D843B1B3F5806F0B
:10383C0019D1002104F10800FFF7A4FB0546002D67
:10384C0049D1734A936D23F4E053D4F898100B4389
:10385C00936516E0022104F12800FFF719FC0546D8
:10386C00BEE72E46D5E7012635460AE0B3F5805F64
:10387C00E5D0B3F5A05FE2D0B3F5406FDFD0012601
:10388C003546216801F080020023134333D0D4F86D
:10389C009C30B3F5804F00F0B28021D843B1B3F522
:1038AC00005F1AD1002104F10800FFF76BFB0546FD
:1038BC00002D40F0AB80564A936D23F46043D4F84E
:1038CC009C100B43936516E0022104F12800FFF7CE
:1038DC00DFFB0546B3E72E46D3E7012635460AE063
:1038EC00B3F5004FE4D0B3F5204FE1D0B3F5C04FA2
:1038FC00DED001263546216801F00802002313436F
:10390C000DD0D4F88030B3F5805F00F08380404A4E
:10391C00536D23F44053D4F880100B435365216846
:10392C0001F01002002313430CD0D4F89430B3F5FB
:10393C00807F79D0364A936D23F44073D4F8941079
:10394C000B439365216801F40022002313430CD030
:10395C00D4F8A030B3F5803F00F08080B3F5003F81
:10396C0072D0002B6AD001263546216801F48022E2
:10397C00002313430DD0D4F88430B3F5001F00F0AE
:10398C008580B3F5401F77D0B3F5801F6FD001262B
:10399C003546216801F480320023134308D0236D8F
:1039AC00002B7CD0B3F5803F00F087800126354694
:1039BC00216801F000520023134340F087802168F6
:1039CC0001F400320023134300F08D80E36FB3F554
:1039DC00807F00F0F78040F28380B3F5007F03D046
:1039EC00B3F5407F40F0EC80002D40F0F180084AA8
:1039FC00536D23F44073E16F0B43536573E0022165
:103A0C0004F12800FFF744FB054651E72E4672E708
:103A1C0000440258022104F12800FFF739FB00286A
:103A2C003FF475AF012672E7022104F12800FFF77D
:103A3C002FFB00283FF47EAF01267BE7002104F129
:103A4C000800FFF79FFA05467DB97D4A936D23F474
:103A5C004033D4F8A0100B43936586E7022104F1A0
:103A6C002800FFF715FB0546EEE72E467DE7744A66
:103A7C00D36A43F40033D3627DB9714A536D23F496
:103A8C004013D4F884100B43536582E7012104F1F1
:103A9C002800FFF7FDFA0546EEE72E4679E7684A5F
:103AAC00D36A43F40033D36275B9654AD36C23F4FB
:103ABC008033216D0B43D3647AE7022104F10800B3
:103ACC00FFF760FA0546EFE72E4671E7022104F195
:103ADC002800FFF7DDFA00283FF471AF01266EE7EE
:103AEC00002B81D00126216801F48012002313439E
:103AFC0006D0534A136D23F00043216F0B4313651B
:103B0C00216801F400120023134306D04C4A136DB4
:103B1C0023F08073A16E0B431365216801F0804282
:103B2C000023134309D0464B1A6922F400421A6150
:103B3C001A69D4F8B4100A431A61216801F00042E2
:103B4C000023134306D03E4AD36C23F04053616DDF
:103B5C000B43D364216801F400020023134307D004
:103B6C00374A536D23F44003D4F888100B43536544
:103B7C006168002201F0010313432BD1616800221C
:103B8C0001F0020313432ED16168002201F00403FB
:103B9C00134331D16168002201F00803134334D17F
:103BAC006168002201F01003134337D161680022D1
:103BBC0001F0200313433AD106B101263046F8BD7B
:103BCC00012690E71E4AD36A43F40033D3620BE715
:103BDC002E4688E7002104F10800FFF7D3F90028EE
:103BEC00CCD00646CAE7012104F10800FFF7CAF958
:103BFC000028C9D00646C7E7022104F10800FFF7E8
:103C0C00C1F90028C6D00646C4E7002104F12800FB
:103C1C00FFF73EFA0028C3D00646C1E7012104F1A4
:103C2C002800FFF735FA0028C0D00646BEE702216F
:103C3C0004F12800FFF72CFA0028BDD00646BBE79C
:103C4C000044025808B5FFF757F9054B1B6AC3F33C
:103C5C000213044AD35C03F01F03D84008BD00BF15
:103C6C0000440258E45100082DE9F0410446864B0B
:103C7C009D6A9E6AC6F30536D86AC0F30010DB6BEA
:103C8C00C3F3CC0300FB03F0FCF7F0FB002E00F0B9
:103C9C00F58005F003050746012D79D0022D00F0C3
:103CAC00CB800DB33046FCF7E1FB01467748FCF7BF
:103CBC00E9FC0546744B986BC0F30800FCF7D6FB87
:103CCC0006464FF064513846FCF728FC0146304656
:103CDC00FCF71CFB4FF07E51FCF718FB0146284605
:103CEC00FCF71CFC054674E0674B1B6813F0200FB7
:103CFC002CD0DFF89481D8F80030C3F3C1036448AA
:103D0C00D840FCF7B3FB05463046FCF7AFFB014649
:103D1C002846FCF7B7FC0546D8F83800C0F3080075
:103D2C00FCF7A4FB06464FF064513846FCF7F6FB53
:103D3C0001463046FCF7EAFA4FF07E51FCF7E6FA02
:103D4C0001462846FCF7EAFB054642E03046FCF704
:103D5C008DFB01464F48FCF795FC05464A4B986B8A
:103D6C00C0F30800FCF782FB06464FF0645138465E
:103D7C00FCF7D4FB01463046FCF7C8FA4FF07E51F5
:103D8C00FCF7C4FA01462846FCF7C8FB054620E0C0
:103D9C003046FCF76BFB01463C48FCF773FC0546D0
:103DAC00394B986BC0F30800FCF760FB06464FF0EC
:103DBC0064513846FCF7B2FB01463046FCF7A6FAD4
:103DCC004FF07E51FCF7A2FA01462846FCF7A6FB01
:103DDC0005462D4EB06BC0F34620FCF747FB4FF069
:103DEC007E51FCF793FA01462846FCF74BFCFCF796
:103DFC00E5FC2060B06BC0F30640FCF737FB4FF0DE
:103E0C007E51FCF783FA01462846FCF73BFCFCF795
:103E1C00D5FC6060B06BC0F30660FCF727FB4FF07D
:103E2C007E51FCF773FA01462846FCF72BFCFCF795
:103E3C00C5FCA060BDE8F0813046FCF717FB0146DD
:103E4C001548FCF71FFC05460F4B986BC0F3080098
:103E5C00FCF70CFB06464FF064513846FCF75EFB52
:103E6C0001463046FCF752FA4FF07E51FCF74EFA01
:103E7C0001462846FCF752FB0546AAE700232360BF
:103E8C006360A360D6E700BF004402580024744A64
:103E9C000090D0030024744C20BCBE4B2DE9F041A3
:103EAC000446864B9D6A9E6AC6F30556D86AC0F3D3
:103EBC0000205B6CC3F3CC0300FB03F0FCF7D6FAD9
:103ECC00002E00F0F58005F003050746012D79D092
:103EDC00022D00F0CB800DB33046FCF7C7FA01463B
:103EEC007748FCF7CFFB0546744B186CC0F3080001
:103EFC00FCF7BCFA06464FF064513846FCF70EFB53
:103F0C0001463046FCF702FA4FF07E51FCF7FEF901
:103F1C0001462846FCF702FB054674E0674B1B681C
:103F2C0013F0200F2CD0DFF89481D8F80030C3F3B5
:103F3C00C1036448D840FCF799FA05463046FCF7B3
:103F4C0095FA01462846FCF79DFB0546D8F840003B
:103F5C00C0F30800FCF78AFA06464FF06451384665
:103F6C00FCF7DCFA01463046FCF7D0F94FF07E51F5
:103F7C00FCF7CCF901462846FCF7D0FA054642E09E
:103F8C003046FCF773FA01464F48FCF77BFB0546BD
:103F9C004A4B186CC0F30800FCF768FA06464FF061
:103FAC0064513846FCF7BAFA01463046FCF7AEF9D4
:103FBC004FF07E51FCF7AAF901462846FCF7AEFA01
:103FCC00054620E03046FCF751FA01463C48FCF728
:103FDC0059FB0546394B186CC0F30800FCF746FA40
:103FEC0006464FF064513846FCF798FA01463046C5
:103FFC00FCF78CF94FF07E51FCF788F90146284606
:10400C00FCF78CFA05462D4E306CC0F34620FCF7BD
:10401C002DFA4FF07E51FCF779F901462846FCF752
:10402C0031FBFCF7CBFB2060306CC0F30640FCF797
:10403C001DFA4FF07E51FCF769F901462846FCF752
:10404C0021FBFCF7BBFB6060306CC0F30660FCF737
:10405C000DFA4FF07E51FCF759F901462846FCF752
:10406C0011FBFCF7ABFBA060BDE8F0813046FCF720
:10407C00FDF901461548FCF705FB05460F4B186C7E
:10408C00C0F30800FCF7F2F906464FF064513846CD
:10409C00FCF744FA01463046FCF738F94FF07E51F4
:1040AC00FCF734F901462846FCF738FA0546AAE72E
:1040BC00002323606360A360D6E700BF004402586E
:1040CC000024744A0090D0030024744C20BCBE4BD6
:1040DC00026852E8003F23F4907342E80031002953
:1040EC00F6D1026802F1080353E8001F0D4B0B4098
:1040FC00083242E800310029F3D1C36E012B06D0FF
:10410C002023C0F88C300023C366436770470268D5
:10411C0052E8003F23F0100342E800310029F6D1A9
:10412C00EEE700BFFEFFFFEF704708B5026852E8EC
:10413C00003F23F0400342E800310029F6D1202350
:10414C00C0F8883000238367FFF7EEFF08BD704787
:10415C0008B5806B0023A0F85E30A0F85630FFF74E
:10416C00F6FF08BD7047000070B504460168CB69C6
:10417C0008688D6840F60F021A4008D113F0200F22
:10418C0005D010F0200F34D115F0805F31D12AB159
:10419C00B34A2A4033D1B34E304230D1E26E012AB9
:1041AC0000F0C68013F4801F03D015F4800F40F08C
:1041BC009B8113F0800F07D010F0800F40F09B8193
:1041CC0015F4000F40F0978113F0400F03D010F05E
:1041DC00400F40F0978113F4000F03D010F0804F84
:1041EC0040F0948113F0807F02D00028C0F29281BD
:1041FC0070BD636F002BFBD020469847F8E713F097
:10420C00010F09D010F4807F06D001260E62D4F87D
:10421C0090103143C4F8901013F0020F0BD015F02E
:10422C00010F08D0216802260E62D4F8901041F0DC
:10423C000401C4F8901013F0040F0BD015F0010F0B
:10424C0008D0216804260E62D4F8901041F00201C7
:10425C00C4F8901013F0080F0BD010F0200F00D101
:10426C003AB1226808211162D4F890200A43C4F8AC
:10427C00902013F4006F0CD010F0806F09D02268DE
:10428C004FF400611162D4F8902042F02002C4F87F
:10429C009020D4F89020002AAAD013F0200F09D037
:1042AC0010F0200F02D115F0805F03D0636F0BB1BB
:1042BC0020469847D4F8902023689B6813F0400F51
:1042CC0002D112F0280F2CD02046FFF701FF2368F3
:1042DC009B6813F0400F20D0226802F1080353E8CA
:1042EC00003F23F04003083242E800310029F3D1AB
:1042FC00D4F880306BB15C4A1A65D4F88000FDF7B5
:10430C0097F900283FF474AFD4F88000036D9847F8
:10431C006EE72046FFF71BFF6AE72046FFF717FF03
:10432C0066E72046FFF713FF0023C4F890305FE7E1
:10433C0013F0100F3FF436AF10F0100F3FF432AF04
:10434C0010230B6223689B6813F0400F00F09280DF
:10435C00D4F880201368454845498B4218BF8342E6
:10436C002DD018318B422AD018318B4227D01831DE
:10437C008B4224D018318B4221D018318B421ED065
:10438C0018318B421BD001F556718B4217D0183166
:10439C008B4214D018318B4211D018318B420ED075
:1043AC0018318B420BD018318B4208D018318B420C
:1043BC0005D018318B4202D05B689BB201E05B6880
:1043CC009BB2002B3FF414AFB4F85C1099427FF60B
:1043DC000FAFA4F85E30D369B3F5807F32D022687A
:1043EC0052E8003F23F4807342E800310029F6D1F3
:1043FC00226802F1080353E8003F23F0010308325E
:10440C0042E800310029F3D1226802F1080353E895
:10441C00003F23F04003083242E800310029F3D179
:10442C002023C4F88C300023E366226852E8003F56
:10443C0023F0100342E800310029F6D1D4F88000B3
:10444C00FCF756FF02232367B4F85C10B4F85E3017
:10445C009BB2C91A89B22046FFF784FEC8E600BF9A
:10446C0001000010200100045D4100081000024012
:10447C0028000240B4F85C10B4F85E309BB2C91A44
:10448C0089B2B4F85E309BB2002B3FF4B1AE002978
:10449C003FF4AEAE226852E8003F23F4907342E83A
:1044AC0000300028F6D1226802F1080353E8000F0F
:1044BC001A4B0340083242E800300028F3D1202385
:1044CC00C4F88C300023E3666367226852E8003F2F
:1044DC0023F0100342E800300028F6D102232367B2
:1044EC002046FFF73FFE83E64FF480130B62204615
:1044FC0000F0F0FC7CE6A36F002B3FF479AE204675
:10450C00984775E62046FFF710FE71E6204600F04E
:10451C00E3FC6DE6204600F0DEFC69E6FEFFFFEFF3
:10452C002DE9F04186B004460168836802691343A3
:10453C0042691343C26913430868914A024013430A
:10454C000B602268536823F44053E1680B435360BB
:10455C00A16922688B4B9A4201D0236A1943906857
:10456C00894B03400B4393602268D36A23F00F03FB
:10457C00616A0B43D3622268844B9A4229D0844BE4
:10458C009A4200F09480834B9A4200F0AA80824BAE
:10459C009A4200F0C080814B9A4200F0D680804B4A
:1045AC009A4200F009817F4B9A4200F02E817E4B9B
:1045BC009A4200F041817D4B9A4200F054817C4B31
:1045CC009A4200F079816F4B9A4200F09E818023D1
:1045DC0033E0784B5B6D03F03803282B65D8DFE8AC
:1045EC0013F029006400640064006400640064003B
:1045FC006400AC0164006400640064006400640046
:10460C0064002B00640064006400640064006400B7
:10461C0064005E0064006400640064006400640074
:10462C006400600064006400640064006400640062
:10463C0064006200012300E0082352498A4200F022
:10464C009581E069B0F5004F00F00D82202B00F24F
:10465C006682202B00F2BA82DFE813F087028D020B
:10466C00B802B8029002B802B802B8029502B802B9
:10467C00B802B802B802B802B802B8029A02B8027C
:10468C00B802B802B802B802B802B802B802B8024E
:10469C00B802B802B802B802B802B802A6021023D7
:1046AC00CBE72023C9E74023C7E78023C5E7414B6D
:1046BC005B6D03F00703052B11D8DFE813F0060040
:1046CC00400108000A000C000E000023B5E7082387
:1046DC00B3E71023B1E72023AFE74023ADE78023F6
:1046EC00ABE7344B5B6D03F00703052B11D8DFE808
:1046FC0013F00600280108000A000C000E0000232D
:10470C009BE7082399E7102397E7202395E740239D
:10471C0093E7802391E7274B5B6D03F00703052B91
:10472C0011D8DFE813F00600100108000A000C0095
:10473C000E00002381E708237FE710237DE7202369
:10474C007BE7402379E7802377E71A4B5B6D03F017
:10475C000703052B11D8DFE813F00600F80008005A
:10476C000A000C000E00002367E7082365E71023FE
:10477C0063E7202361E740235FE780235DE700BF09
:10478C00F369FFCF000C0058FFF4FF11001001403B
:10479C000044004000480040004C004000500040E5
:1047AC000014014000780040007C004000180140DB
:1047BC00001C014000440258694B5B6D03F0380348
:1047CC00282B20D8DFE803F0151F1F1F1F1F1F1FEA
:1047DC00C31F1F1F1F1F1F1F171F1F1F1F1F1F1F41
:1047EC00191F1F1F1F1F1F1F1B1F1F1F1F1F1F1FD7
:1047FC001D00012321E708231FE710231DE72023B9
:10480C001BE7402319E7802317E7554B5B6D03F03B
:10481C000703052B0ED8DFE803F0039C0507090BF3
:10482C0000230AE7082308E7102306E7202304E700
:10483C00402302E7802300E7494B5B6D03F007033D
:10484C00052B0ED8DFE803F003870507090B0023BF
:10485C00F3E60823F1E61023EFE62023EDE64023F0
:10486C00EBE68023E9E63E4B5B6D03F03803282B27
:10487C0020D8DFE803F0151F1F1F1F1F1F1F721FFB
:10488C001F1F1F1F1F1F171F1F1F1F1F1F1F191F3A
:10489C001F1F1F1F1F1F1B1F1F1F1F1F1F1F1D0041
:1048AC000123CAE60823C8E61023C6E62023C4E683
:1048BC004023C2E68023C0E6294B5B6D03F038032E
:1048CC00282B20D8DFE803F0151F1F1F1F1F1F1FE9
:1048DC004E1F1F1F1F1F1F1F171F1F1F1F1F1F1FB5
:1048EC00191F1F1F1F1F1F1F1B1F1F1F1F1F1F1FD6
:1048FC001D000123A1E608239FE610239DE620233B
:10490C009BE6402399E6802397E603F50E339B6DD7
:10491C0003F00703052B0ED8DFE803F00326050789
:10492C00090B022389E6082387E6102385E620235A
:10493C0083E6402381E680237FE604237DE604237F
:10494C007BE6042379E6042377E6042375E6042347
:10495C0073E6042371E604236FE604236DE600BFBF
:10496C0000440258042368E6042366E6202B27D86B
:10497C00022BC0F01D81023B1E2B00F21B81DFE8D5
:10498C0013F05200190158001901190119015D00A9
:10499C0019011901190119011901190119016200F3
:1049AC00190119011901190119011901190119012B
:1049BC0019011901190119011901190119016E00C7
:1049CC00402B2ED14FF40040626A824B33F81220F8
:1049DC00B0FBF2F3656805EB4501994200F2EC80FF
:1049EC00B3EB053F00F2EA804FF0000892B20023CF
:1049FC004146FBF703FF0F0247EA106706026808FF
:104A0C002A464346301847F10001FBF7F7FEA0F5A4
:104A1C004072714B9A4200F2D3802368D8604046B2
:104A2C0098E0012096E0FFF70DF90028CCD100208A
:104A3C0090E003A8FFF718F90498F6E76846FFF72B
:104A4C002DFA0198F1E7654B1B6813F0200F08D085
:104A5C00624B1B68C3F3C1036148D840E5E761486A
:104A6C00B2E75F48B0E7202B15D8202B00F2AA80C4
:104A7C00DFE803F03238A8A83BA8A8A840A8A8A84B
:104A8C00A8A8A8A845A8A8A8A8A8A8A8A8A8A8A8FD
:104A9C00A8A8A8A85100402B1CD1626A4D4B33F832
:104AAC001230B0FBF3F06268530803EB4000B0FB2C
:104ABC00F2F0A0F110024FF6EF739A4200F28480EC
:104ACC0083B223F00F03C0F3420018432368D8606D
:104ADC0000203FE001203DE0FEF730FA0028DCD159
:104AEC00002037E0FEF73CFAF8E703A8FFF7BCF824
:104AFC000498F3E76846FFF7D1F90198EEE7374BD6
:104B0C001B6813F0200F08D0344B1B68C3F3C10390
:104B1C003348D840E2E73348BFE73148BDE7402B84
:104B2C0017D14FF40040626A2A4B33F81230B0FBB5
:104B3C00F3F0636800EB5300B0FBF3F0A0F110024C
:104B4C004FF6EF739A4243D8236880B2D8600020A6
:104B5C0000E001200123A4F86A30A4F86830002397
:104B6C006367A36706B0BDE8F081FEF7E7F900289C
:104B7C00D9D10020EEE7FEF7F3F9F8E703A8FFF729
:104B8C0073F80498F3E76846FFF788F90198EEE7A5
:104B9C00124B1B6813F0200F08D0104B1B68C3F38B
:104BAC00C1030F48D840E2E70E48BCE70C48BAE70F
:104BBC000120CFE70120CDE70120CBE70120C9E799
:104BCC000120C7E70120C5E70120C3E70120C1E7A9
:104BDC000120BFE704520008FFFC0F0000440258FC
:104BEC000090D00300093D00836A13F0080F06D033
:104BFC000268536823F40043816B0B435360836A50
:104C0C0013F0010F06D00268536823F40033C16A15
:104C1C000B435360836A13F0020F06D0026853688B
:104C2C0023F48033016B0B435360836A13F0040F3E
:104C3C0006D00268536823F48023416B0B43536006
:104C4C00836A13F0100F06D00268936823F4805324
:104C5C00C16B0B439360836A13F0200F06D002687C
:104C6C00936823F40053016C0B439360836A13F035
:104C7C00400F0AD00268536823F48013416C0B4335
:104C8C005360436CB3F5801F0BD0836A13F0800F15
:104C9C0006D00268536823F40023C16C0B435360A5
:104CAC0070470268536823F4C003816C0B43536054
:104CBC00EBE72DE9F84305460E4617469946DDF815
:104CCC0020802C68E46936EA04030CBF012400241C
:104CDC00BC423AD1B8F1FF3FF3D0FCF79BFAA0EB02
:104CEC000900404534D8B8F1000F33D02B681A684E
:104CFC0012F0040FE5D0B6F1400218BF0122802E4D
:104D0C00DFD0002ADDD0DA6912F0080F11D1DA6990
:104D1C0012F4006FD5D04FF400621A622846FFF7E8
:104D2C00D7F92023C5F89030002385F88430032070
:104D3C000CE008241C622846FFF7CAF9C5F890401D
:104D4C00002385F88430012000E00020BDE8F883C2
:104D5C000320FBE70320F9E730B583B004460023BA
:104D6C00C0F89030FCF756FA054623681B6813F020
:104D7C00080F10D123681B6813F0040F28D12023CF
:104D8C00C4F88830C4F88C300020E066206784F8C2
:104D9C00840003B030BD6FF07E43009303460022C5
:104DAC004FF400112046FFF784FF0028E2D0226860
:104DBC0052E8003F23F0800342E800310029F6D18D
:104DCC002023C4F88830002384F884300320E0E7E3
:104DDC006FF07E4300932B4600224FF48001204657
:104DEC00FFF767FF0028CAD0226852E8003F23F47F
:104DFC00907342E800310029F6D1226802F10803D1
:104E0C0053E8003F23F00103083242E80031002947
:104E1C00F3D12023C4F88C30002384F88430032091
:104E2C00B7E778B310B50446D0F888300BB3242319
:104E3C00C4F888302268136823F001031360A36A56
:104E4C00E3B92046FFF76CFB012811D022685368A8
:104E5C0023F4904353602268936823F02A039360F1
:104E6C002268136843F0010313602046FFF774FFB8
:104E7C0010BD80F88430FCF7EBF8D8E72046FFF73C
:104E8C00B3FEDEE701207047436E2BB90123A0F877
:104E9C006A30A0F86830704730B403689A68C2F37F
:104EAC0042629968490F094D6B5C1B01084C615CAF
:104EBC0093FBF1F3A0F86A30AB5C1B01A25C93FB93
:104ECC00F2F3A0F8683030BC704700BF24520008E1
:104EDC001C52000870477047704790F88430012BC3
:104EEC0018D0012380F884302423C0F8883003685C
:104EFC001A68196821F00101196022F00052002390
:104F0C00436601680A602022C0F8882080F884304B
:104F1C00184670470220704738B590F88430012B42
:104F2C001DD00446012380F884302423C0F8883037
:104F3C0003681D681A6822F001021A6002689368FF
:104F4C0023F0604319439160FFF79EFF23681D60B7
:104F5C002023C4F88830002084F8840038BD022057
:104F6C00FCE738B590F88430012B1DD004460123A2
:104F7C0080F884302423C0F8883003681D681A68D0
:104F8C0022F001021A600268936823F060631943EF
:104F9C009160FFF779FF23681D602023C4F88830E7
:104FAC00002084F8840038BD0220FCE770B50D4E5B
:104FBC000D4D761BB61006D0002455F8043B013479
:104FCC009847A642F9D1094E094D761B00F0D2F84C
:104FDC00B61006D0002455F8043B01349847A6427D
:104FEC00F9D170BD38520008385200084052000800
:104FFC0038520008F0B4860746D0541E002A3CD024
:10500C00CAB2034601E0013C37D303F8012B9D07DC
:10501C00F9D1032C2AD9CDB245EA05250F2C45EA46
:10502C00054534D9A4F1100222F00F0C03F120072E
:10503C001609674403F1100242E9045542E902558E
:10504C001032BA42F8D1721C14F00C0F03EB02129E
:10505C0004F00F0613D0331F23F00303043313445F
:10506C0042F8045B9342FBD106F003042CB1CAB2A4
:10507C001C4403F8012B9C42FBD1F0BC7047344616
:10508C001346002CF3D1F8E714460346C1E71A4641
:10509C002646E0E7024B13B1024800F005B8704712
:1050AC0000000000C1500008002301461A461846B3
:1050BC0000F01AB838B5084B084D5B1B9C1007D094
:1050CC00043B1D44013C55F804399847002CF9D198
:1050DC00BDE8384000F054B8445200084052000873
:1050EC00704700BF704700BF2DE9F047DFF880A084
:1050FC000646DAF8000098460F469146FFF7F0FF97
:10510C001A4B1B68D3F8484124B365681F2D26DC65
:10511C005EB9AB1C0135DAF80000656044F8237009
:10512C00FFF7E0FF0020BDE8F08704EB85030121C9
:10513C00C3F88890D4F88821A9400A43022EC4F8F9
:10514C008821C3F80881E4D1D4F88C311943C4F810
:10515C008C11DEE703F5A674C3F84841D5E7DAF8FD
:10516C000000FFF7BFFF4FF0FF30DCE72C520008C8
:10517C0038040024F8B500BFF8BC08BC9E46704744
:0C518C00F8B500BFF8BC08BC9E46704798
:105198000000000000000000000000000000000007
:1051A80000000000010000000200000003000000F1
:1051B80004000000000000000500000000000000DE
:1051C80000000000000000000600000000000000D1
:1051D80000000000000000000700000000000000C0
:1051E800010203040102030406070809000102037F
:1051F80004050607080C10141820304001000200AE
:105208000400060008000A000C00100020004000FE
:1052180080000001080402040801010101010103E2
:08522800070100001000002442
:0852300008B6FF7F0100000039
:08523800A1500008F10200087A
:04524000CD02000893
:105244000090D0030090D003010000001000000083
:1052540000000000FC02002464030024CC030024AA
:10526400000000000000000000000000000000003A
:10527400000000000000000000000000000000002A
:10528400000000000000000000000000000000001A
:10529400000000000000000000000000000000000A
:1052A40000000000000000000000000000000000FA
:1052B40000000000000000000000000000000000EA
:1052C40000000000000000000000000000000000DA
:1052D40000000000000000000000000000000000CA
:1052E40000000000000000000000000000000000BA
:1052F40000000000000000000100000000000000A9
:105304000E33CDAB34126DE6ECDE05000B0000006D
:105314000000000000000000000000000000000089
:105324000000000000000000000000000000000079
:105334000000000000000000000000000000000069
:105344000000000000000000000000000000000059
:0C56740000000000000000009805002469
:0400000508001109D5
:00000001FF
